:1000000018C017C016C015C014C013C012C04FC00E
:1000100010C00FC00EC0969860E06FBD60E06DBD6F
:100020006CBD66E06EBDEBD0549A5F9BFCCF3FC0C9
:1000300036C06FED6DBF69E169B960E462BB60E431
:1000400061BB68E3662E60E0762EA0E095D051C0DB
:10005000BAE373D0B0E271D0B0E26FD074D0AF33F6
:1000600011F1AD3029F3A13211F1AF7DBA2F65D076
:10007000B0E263D062D0A23591F0AD34E1F0A435A6
:1000800051F2A134F1F0A23441F1A33491F1A4343E
:10009000E1F1A534A9F0A03521F05FD0D9CF90D0FF
:1000A000D7CF44C1D5CFF4E0E0E35BD0D1CFA89562
:1000B00068E061BDFFCF84D0549A5F9BFCCFF7CF3F
:1000C00030C061E0262E61E0362E64EF462E67E2F6
:1000D000562EF4E0E8EF45D0BBCF61E0262E6AE073
:1000E000362E64EF462E67E2562EF5E0E4E239D074
:1000F000AFCF61E0262E64E6362E64EF462E67E22F
:10010000562EF5E0EEE42DD0A3CF6AE0262E64E66D
:10011000362E64EF462E67E2562EF5E0E4E721D056
:1001200097CF64E6262E64E6362E64EF462E67E20D
:10013000562EF5E0EEE915D08BCF539A5D9BFDCF9F
:10014000BCB953980895549A5F9BFDCFACB15498B5
:100150000895F9DFBA2FF1DF0895F4E0E4EF01D05C
:100160000895C895002021F0B02DE7DF3196F9CF32
:100170000895F7DFF2DF0895F0DFEFDFF3E0E2EC60
:10018000F8DF08954C2F4695469546954695405D77
:100190004A3308F0495FCF70C05DCA3308F0C95FC9
:1001A0000895F0DFB42FC9DFBC2FC7DF089568E0E2
:1001B000B0E3CC1F08F4B1E3C0DF6A95C9F7089536
:1001C00060E96AB9789460E06FBD60E06DBD6CBDB8
:1001D00066E06EBD122C9698932D742D852D7A9520
:1001E0007030E9F78A958030D1F7000000009A95C9
:1001F000A1F71A9489F760E06EBDF894969A0CB551
:100200001DB50CD0AADFBF2D60E3B60F96DFCE2D53
:10021000C8DFCD2DC6DFB0E290DF089520E1FF24D6
:10022000EE24DD24FF27000F111FDD1CEE1CFF1C38
:100230002A9509F40895E0E132913D5F33FD308362
:100240003081305D37FD3083ED30B1F7ECCF5D9B11
:10025000FECFC895002009F40895C8950CB83196D2
:10026000F6CF25CF22243324969A5F9BFDCF0CB185
:100270000CB90636B1F30634A1F3013431F101367D
:1002800021F10D30E1F0005310F00A3028F0E4E1E4
:10029000F6E0DDDF08940895422C532C220C331C29
:1002A000B0F3220C331C98F3240C351C80F3220C81
:1002B000331C68F35524200E351C48F3D5CF5D9BC5
:1002C000FECF0AE00CB988940895E8EEF5E0BFDFB0
:1002D0005F9BFECF0CB160E26CB90F7D0CB90134AD
:1002E00061F0023469F0033471F0043479F00534BC
:1002F00081F0063489F0073491F068E0662E12C070
:1003000060E1662E0FC068E1662E0CC060E2662ECA
:1003100009C068E2662E06C060E3662E03C068E38B
:10032000662E00C0ECECF5E092DF00C00FED0DBFD3
:1003300060E462BB68E761BB09E109B908E10AB999
:10034000F6E0EAED84DFF6E0E2E681DF8BDFD8F36A
:10035000222D332D022D032911F428EA31E6F6E08F
:10036000E6E375DF7FDFD8F3422D532D022D0329FD
:1003700011F440ED57E0A42FB52F159720F31196F7
:100380002A2E3B2EC22FD32FCA1BDB0BE0F2259760
:10039000D0F221964C2E5D2EF6E0EEE858DF9698CE
:1003A000000062BA1197F1F75F99CDCF000072BAE1
:1003B0002197F1F7A22DB32DC42DD52D00000000FB
:1003C000EFCF4672657175656E6379206D657465F2
:1003D000722F70756C73652067656E657261746FDE
:1003E0007220323030322E30322E30392072657623
:1003F0002E420A0D4672657175656E6379206D65D2
:1004000074657220284329323030322062792052BC
:100410006963686172642043617070656C732C61FC
:1004200076724063617070656C732E6F72672E20F8
:100430000A0D413D31306D732C423D3130306D73CA
:100440002C433D31732C443D3130732C453D3130CC
:1004500030732E200A0D523D72656164206672650C
:10046000712E204D3D636F6E74696E756F757320CC
:10047000667265712E20542D72756E6E696E6720DE
:10048000746F74616C2E0A0D5020746F207377693D
:1004900074636820746F2070756C73652067656E77
:1004A000657261746F722C20213D726573657420D2
:1004B0000A0D4D617820636F756E743D20363535B9
:1004C00033362C204D6178206672657175656E63D8
:1004D000793C20344D20487A2E204E6F206F76656F
:1004E00072666C6F7720646574656374696F6E2ED5
:1004F0000A0D0A0D0A0D000054696D65626173658D
:100500003D203130206D732E204672657175656E09
:1005100063793D20436F756E7420583130302E2042
:100520000A0D000054696D65626173653D203130CC
:1005300030206D732E204672657175656E63793D4E
:1005400020436F756E74205831300A0D00005469D5
:100550006D65626173653D203120732E20467265A2
:100560007175656E63793D20436F756E74205831E7
:100570000A0D000054696D65626173653D2031307C
:1005800020732E204672657175656E63793D204338
:100590006F756E742058312F31300A0D0000546988
:1005A0006D65626173653D2031303020732E2046C9
:1005B00072657175656E63793D20436F756E742049
:1005C00058312F31303020200A0D000020202A2AF7
:1005D00050756C736520616D706C6974756465200D
:1005E0007365742E0A0D00000A0D456E7465722045
:1005F000616D706C697475646520412E2E472028EA
:1006000064656661756C743D20472C6D6178292E98
:10061000202000004572726F7220696E20696E7032
:1006200075742E2052657065617420696E707574E2
:100630002E200D0A0000496E707574206163746984
:1006400076652074696D652C2041206F72204620EC
:100650002864656661756C743D322C303030293AFF
:100660000000496E707574206379636C652074694D
:100670006D652C2041206F722046202864656661DC
:10068000756C743D32352C303030293A0000436FA0
:100690006E74696E756564206F7065726174696FE0
:1006A0006E2E456E746572206E6577206379636C7B
:1006B00065206C656E67746820746F2073746F704A
:1006C00020616E6420726573746172742067656E58
:1006D000657261746F720D0A00000A0D0A0D5055A3
:1006E0004C53452047454E455241544F522E2028E9
:1006F00043293230303020627920696E666F406164
:1007000076722D61736D2D7475746F7269616C2EC4
:100710000A0D544F2052455455524E20544F2046F6
:1007200052455155454E4359204D455445522C2074
:10073000454E5445522046204B45592E20200D0A47
:10074000466F722070756C736520616D706C697492
:10075000756465206D656E752C20707265737320ED
:10076000412E0A0D416C6C2074696D6573206973AC
:1007700020696E206D6963726F2D7365636F6E649F
:10078000732C2074686520616363657074656420F0
:1007900072616E676520697320352E2E36353533CC
:1007A000352E0D0A4E65772076616C756520737461
:1007B0006F7073206F7065726174696F6E20756EF3
:1007C00074696C20616C6C20696E7075742069733B
:1007D00020636F6D706C657465642E200A0D0A0AC3
:1007E0000000FFFFFFFFFFFFFFFFFFFFFFFFFFFF17
:1007F000FFFFFFFFFFFFFFFFFFFFFFFFFFFFFFFF09
:00000001FF
